:020000040000FA
:020000000428D2
:08000800FF30A200FF30A3004D
:10001000FF30A400FF30A5000F30A600AC01AD01F9
:10002000AE01AF01B001A01400308A110A12EA201B
:1000300000308A110A12E62000308A110A12E220EA
:1000400000308A110A12DE2000308A110A12D320F1
:100050002C08B10005308A110A1273203108AC0057
:100060002D08B10007308A110A1273203108AD0043
:100070002E08B10007308A110A1273203108AE0031
:100080002F08B10007308A110A1273203108AF001F
:100090003008B10002308A110A1273203108B00012
:1000A0002C08FF3A8A110A12C0202D08FF3A8A1143
:1000B0000A12BC202E08FF3A8A110A12B8202F0813
:1000C000FF3A8A110A12B4203008FF3A8A110A1244
:1000D000B02001308A110A128D208A110A122828B4
:1000E0008A110A127028B2003108B5003208B60031
:1000F0008A110A120D213708B4003408B300031026
:10010000B10D8A110A12A01C8628B10AA0108A110A
:100110000A12331C8C28A0140800B1003108B20068
:100120006430B3000A308A110A129628B400FF30F6
:10013000B5003308B7003208B60077308A110A12CA
:1001400035070318A0288A110A12B60B9D288A11B8
:100150000A12B70B9B288A110A12B40B99280800BF
:10016000AB008A110A12C428AA008A110A12C728F1
:10017000A9008A110A12CA28A8008A110A12CD28D9
:10018000A7008A110A12D0282B08890008002A0823
:100190008800080029088700080028088600080051
:1001A000270885000800B10031080F39B200260881
:1001B000F0393204A6008A110A12EE28A5008A112D
:1001C0000A12F628A4008A110A12FE28A3008A1136
:1001D0000A120129A2008A110A12042926088A118A
:1001E0000A12072189008A110A120A2925088A1190
:1001F0000A12072188008A110A120A2924086700B6
:10020000080023086600080022086500080083161D
:10021000031308008312031308003608003C8A11F8
:100220000A12031C16298A110A121E290310B50C82
:1002300001303602B6008A110A120D293508B700BE
:020240000800B4
:02400E00723FFF
:00000001FF
